:1000000000308A0021290000FF00030E8301A600B2
:100010007F08A5000A08AD008A01A50E0408A70004
:100020002008A8002108A9002208AA002308AB0084
:100030002408AC00831383128C308400801E222895
:100040008C1A3528270884002808A0002908A10058
:100050002A08A2002B08A3002C08A4002D088A005F
:10006000260E8300FF0E7F0E09008A1178280A10E1
:100070008A100A1182074C3469346134693473344C
:100080006F346E3420344F344B3400340A108A10ED
:100090000A118207503441345334203442344F34EF
:1000A0004E343E340034A001A1014208031043182D
:1000B000A007A00CA10CC318A007A00CA10C431909
:1000C000A007A00CA10CC319A007A00CA10C431AF7
:1000D000A007A00CA10CC31AA007A00CA10C431BE5
:1000E000A007A00CA10CC31BA007A00CA10C0034FE
:1000F00083128C122E0BA2288C1E7C281A08B100A9
:100100003108443C031994283108473C03199428CA
:100110003108423C031994283108413C03199428C2
:100120003108433C031D9F280130AE073108433C92
:10013000031D9E280130AE00B5000B29A128013017
:10014000B6000B292E08023C031DC5288C1EA628CC
:100150001A08B20032082F3C0318B2283208393C82
:100160000318B6280130AE00B600C5280130AE072E
:100170003108413C031DC4280130AE00303032024A
:10018000B0000130B5000B290B292E08033C031DDC
:10019000DC288C1EC9281A08B30033082F3C03182A
:1001A000D5283308393C0318D9280130AE00B600F1
:1001B000DB280130AE070B292E08043C031D0B2958
:1001C0008C1EE0281A08B40034082F3C0318EC28D1
:1001D0003408393C0318F0280130AE00B6000A2973
:1001E0000130AE00B50030303202BE00C2006430D3
:1001F000C30053202108BF0030303302C100C200C9
:100200000A30C300532021083F07C20030303402B7
:100210004207AF000B298C128A1122283C3084003F
:100220000008031920290630A100A001A00B1629FF
:10023000A10B15297B30A000A00B1C29800B1329D2
:10024000003484011F30830583161F149F141F156B
:100250009F1107309C001C0883120D134030831639
:10026000990026309800903083129800AF01B001B9
:10027000B501FF30BA000230BB00FA30BC000E21DD
:10028000BB0B3D29BB013B083720BB0AA00020085F
:100290000C1E482999000A303B02031D43290D30EA
:1002A0000C1E502999000A300C1E542999003E302A
:1002B0000C1E5829990000308316850086008500A1
:1002C0008312850183168600831286010430BB00E9
:1002D000FA30BC000E21BB0B68290130AE00B5011D
:1002E0003A113A0883168700831207110C309700E1
:1002F000BA103A0883168700831287100C309D00CD
:100300000030A10006389200FF308316920083125D
:1003100095019B010230BB00FA30BC000E21BB0BE3
:100320008C29831686108312861083160611831279
:100330000615831686118312861183160612831200
:10034000061683128C1283168C16C03083128B040F
:10035000360BC0290D300C1EAB2999000A300C1E3B
:10036000AF299900BB013B084620BB0AA00020082A
:100370000C1EB829990008303B02031DB329B601B1
:10038000350B9B2A0D300C1EC32999000A300C1E18
:10039000C72999004F300C1ECB2999004B300C1EF9
:1003A000CF2999003E300C1ED3299900AF080319BC
:1003B000E3292F08633C031CE3293108413C03195E
:1003C000E3296430AF003108443C031DED292F08B8
:1003D000B700390BED29370895003108433C031D60
:1003E000F42995019B01B9013108473C031DFE2901
:1003F0002F08B800390BFE2938089B003108423C11
:10040000031D0C2A2F08B7002F08B800390B0C2A3F
:100410003708950038089B003108413C031D9A2A93
:10042000300B1A2A83168610831286108316061143
:10043000831206153008023C031D262A8316061176
:100440008312061183168610831286143008033C2B
:10045000031D322A83168611831286118316061213
:10046000831206163008043C031D3E2A831606122A
:100470008312061283168611831286153008053CF6
:10048000031D522A831686108312861083160611C6
:10049000831206158316861183128611831606129F
:1004A000831206163008063C031D662A83160611C1
:1004B0008312061183168610831286148316061281
:1004C0008312061283168611831286153008073CA4
:1004D000031D7A2A8316861083128610831606114E
:1004E00083120615831606128312061283168611CE
:1004F000831286153008083C031D8E2A83160611C8
:1005000083120611831686108312861483168611B1
:100510008312861183160612831206163008083CD1
:100520000318942A0130B6003708950038089B005C
:0A0530000130B900B501A8296300ED
:02400E00323F3F
:00000001FF
